:100000000C9463020C94AA020C94AA020C94AA0207
:100010000C94AA020C94AA020C94AA020C94AA02B0
:100020000C94AA020C94AA020C94FF0B0C94D10C11
:100030000C94AA020C94AA020C94AA020C94AA0290
:100040000C94AA020C9445210C94AA020C94AA02C6
:100050000C94AA020C94D71A0C94AA020C94AA022B
:100060000C94AA020C94AA020C94AA020C94AA0260
:100070000C94AA020C94AA020C94AA020C94AA0250
:100080000C94AA020C94AA020C94AA020C94AA0240
:100090000C94AA020C94AA020C94AA020C94AA0230
:1000A0000C94AA020C94AA020C94AA023E0D600DB4
:1000B000530E600D530EA50DC80D530E1D0E300EC0
:1000C0001A111A11491149118C11C611D313D313E6
:1000D000DF11D313D412D412A713D313D313BE1327
:1000E00029002B00E000E100357100001E00140023
:1000F00004001D006400E3001F001A0016001B002E
:1001000000000252200008000700060000002C003A
:100110002100150009001900E2001151220017000A
:100120000A0005000000460023001C0000000B0030
:100130000000650023000A000000050000004800E0
:1001400024001C000B0011000000007525001800A1
:100150000D001000E600115126000C000E003600C4
:1001600000002C00270012000F0037002F00015262
:100170002D001300330038003000E7002A0028006B
:100180002800E500347100000100010001000100B9
:100190000100000001001E022002220201000100F5
:1001A00001001F02210223020100010001002F02B1
:1001B00026022F000100010001003002270230005A
:1001C000010012510100310235003502000001002A
:1001D0000100010000000100000001000100010019
:1001E0000000010000000100010001000100010009
:1001F0000000010000005F005C0059006200125125
:10020000540060005D005A0062000100550061006A
:100210005E005B0063000100560057005700580065
:10022000580001002E0032003400010001000000DF
:100230000100010001000100010000003A004A0035
:100240005000F400F20001003B0052005100F000A9
:10025000F10001003C004D004F00F500F3000100EB
:100260003D0049004C000100010010513E004B00D0
:100270004E0001000000A5003F0001000000010049
:1002800000004C05400001000000010000000100DA
:1002900041000100010001000000010042000100D6
:1002A000B600AC00AA001051430049004C00AE005B
:1002B000A800010044000100B700AB00A900010044
:1002C00045000100010001000100010001000100E2
:1002D00001000100010000001603450072006700E4
:1002E0006F0044006F007800200045005A000000B5
:1002F00016034500720067006F0044006F0078002D
:10030000200045005A0000000403090409026D00A2
:10031000040100A0FA090400000103010100092101
:1003200011010001223F000705810308000A0904AA
:1003300001000103010200092111010001224D0009
:100340000705820308000A090402000103000000F7
:100350000921110100012236000705830308000A64
:10036000090403000103000000092111010001221A
:10037000390007058403100001120110010000007C
:1003800008EDFE071301000102000105010906A1A5
:1003900001050719E029E715002501950875018178
:1003A0000205081901290595057501910295017548
:1003B0000391010507190029771500250195787526
:1003C000018102C005010980A101850216010026F4
:1003D000B7001A01002AB700751095018100C00509
:1003E0000C0901A1018503160100269C021A0100D7
:1003F0002A9C02751095018100C005010902A10126
:100400000901A10005091901290515002501950516
:1004100075018102950175038101050109300931DA
:100420001581257F95027508810609381581257F7C
:10043000950175088106050C0A38021581257F95FE
:100440000175088106C0C005010906A1010507194B
:10045000E029E715002501950875018102950175D0
:100460000881010508190129059505750191029575
:1004700001750391010507190029FF150025FF9556
:100480000675088100C000000000000000000000A8
:1004900000010204060A0F17202C3A4A5D71879D5D
:1004A000B3C7DAE9F5FCFFFCF5E9DAC7B39D87715C
:1004B0005D4A3A2C20170F0A0604020100000000D2
:1004C00000000000000011241FBECFEFDAE0DEBF05
:1004D000CDBF04B603FE27C08091F1019091F201D7
:1004E000A091F301B091F4018730904BA740B04B3D
:1004F000D1F41092F1011092F2011092F3011092D6
:10050000F40114BE84B7877F84BF0FB6F894A89512
:1005100080916000886180936000109260000FBE3F
:10052000E0E0FFE3099511E0A0E0B1E0ECE2F6E4E1
:1005300002C005900D92A433B107D9F721E0A4E3DE
:10054000B1E001C01D92A13FB207E1F70E94460948
:100550000C9414230C94000061110BC0FC018281E7
:10056000882321F085EE0E94B40F03C085EE0E941F
:100570007C1080E090E0089508956091B50170913D
:10058000B6018091B7019091B8010E94041A569863
:100590005E98E5E3F1E065E070E031E0A1E0B0E015
:1005A0004081831305C091E04F3F41F490E006C0C5
:1005B00021E0411101C020E0922F9195940F90838A
:1005C000992309F194B1AD01062E01C0440F0A949C
:1005D000EAF7942B94B995B1492B45B9408150E085
:1005E000313029F4509389004093880019C032308B
:1005F00029F450938B0040938A0012C050938D00D1
:1006000040938C000DC094B1AD01062E01C0440F83
:100610000A94EAF74095942394B995B1492345B9D2
:100620003F5F6F5F7F4F3196343009F0B9CF089547
:100630000C94BD0256985E9825982D9826982E9871
:1006400027982F988FEF90E09093890080938800EF
:1006500090938B0080938A0090938D0080938C0000
:10066000259A2D9A2FEF80E792E02150804090400C
:10067000E1F700C00000269A2E9A2FEF80E792E063
:10068000215080409040E1F700C00000279A2F9A47
:100690002FEF80E792E0215080409040E1F700C0CA
:1006A000000025982D982FEF80E792E021508040A0
:1006B0009040E1F700C0000026982E982FEF80E7C9
:1006C00092E0215080409040E1F700C00000279860
:1006D0002F9856985E9825982D9826982E982798AA
:1006E0002F98089589EA8093800089E080938100A3
:1006F00024982C983F988AB18F748AB96E98479A3B
:100700008BB1806B8BB9769A0E941A030C94BC0251
:1007100080E2809300018091380181110EC00E9417
:10072000D70381E0809338012FEF83ED90E32150D0
:1007300080409040E1F700C0000080E40E94DD03AB
:100740008093000181112EC00E9407048093000154
:10075000811128C00E94070480930001811122C0EA
:100760008FE30E9407048093000181111BC00E9447
:10077000FF0380E40E94DD0380930001811112C019
:100780008CE00E9407048093000181110BC00E943D
:10079000070480930001811105C08FE30E940704C4
:1007A000809300010E94FF03809100010895109240
:1007B000B9008AE08093B800089594EA9093BC0051
:1007C0009091BC0097FFFCCF9091B900987F983032
:1007D00021F0903111F081E008958093BB0084E80E
:1007E0008093BC008091BC0087FFFCCF8091B90052
:1007F000887F883111F0803471F780E0089584E9B2
:100800008093BC008091BC0084FDFCCF0895809350
:10081000BB0084E88093BC008091BC0087FFFCCFC4
:100820009091B900987F81E0983209F480E00895B2
:1008300084E88093BC008091BC0087FFFCCF80914E
:10084000BB00089580910001811115C080E40E94D1
:10085000DD038093000181110CC082E10E94070436
:1008600080930001811105C08FEF0E9407048093DF
:1008700000010E94FF0384B1807F84B985B1807F2D
:1008800085B98AB1837F8AB98BB1837F8BB93E9852
:10089000469808950E948803809300010E942204D4
:1008A00080B38C7080BB81B3836F81BBE8E4F1E0DF
:1008B000AAE3B1E011921D9281E0E635F807D1F785
:1008C0000C9472039F92AF92BF92CF92DF92EF92FD
:1008D000FF920F931F93CF93DF93809100018823A2
:1008E00079F0809139018F5F80933901811108C0BF
:1008F0000E94880380930001811102C00E941A03A4
:100900008AE3E82E81E0F82E8701C0E0D0E0BB2426
:10091000B39492E0A92ECC24C394D12CC730D10536
:1009200000F580910001811164C080E40E94DD0324
:1009300080930001811112C082E10E94070480931C
:10094000000181110BC0C6010C2E01C0880F0A9452
:10095000EAF780950E940704809300010E94FF033C
:1009600048C0CA30A1F028F4C83059F0C93061F04D
:1009700005C0CC3089F070F0CD3089F0209A2898ED
:1009800010C0219A29980DC0229A2A980AC0239A49
:100990002B9807C0529A01C0539A5B9802C03E9AA6
:1009A0004698E0EAEA95F1F78FB181708B25799945
:1009B00002C032E001C030E0832B7C9902C034E0F9
:1009C00001C030E0832B7D9902C028E001C020E007
:1009D000822B7E9902C090E101C090E0892B9FB1EB
:1009E0009095991F9927991F9295990F907E892B21
:1009F0000FC08091000181114AC080E40E94DD0394
:100A000080930001882381F1912C0E94FF03892D9E
:100A1000D8019C91981719F08C93A09201010E9423
:100A2000220421960F5F1F4FCE30D10509F076CFFB
:100A300080910101882369F181508093010188230D
:100A400039F0EFE9FFE03197F1F700C0000021C075
:100A5000E8E4F1E0D7018D917D018193B8E4EB16D4
:100A6000B1E0FB06B9F715C083E10E94070480934B
:100A700000018111C9CF81E40E94DD038093000150
:100A80008111C2CF0E941804982E9094BECF80E0AE
:100A9000BFCF0E94180381E0DF91CF911F910F918A
:100AA000FF90EF90DF90CF90BF90AF909F90089510
:100AB000E82FF0E0E85BFE4F8081089508958B3BBE
:100AC000910580F4883A910548F5853A9105D8F466
:100AD0008430910508F0B2C0019709F06EC081E042
:100AE00090E00895803E910508F467C0883E910526
:100AF00008F4A4C09C01205F31092031310508F0C1
:100B00005CC090650895853A910509F459C0863A0C
:100B1000910509F058C082E890E40895883A91055B
:100B200009F454C0893A910509F453C08A3A9105F1
:100B300009F452C08B3A910509F451C08C3A9105E1
:100B400009F450C08D3A910509F44FC0803B9105DE
:100B500009F44EC08E3A910509F44DC08F3A9105C3
:100B600009F44CC0813B910509F44BC0823B9105CF
:100B700009F44AC0833B910509F449C0843B9105BF
:100B800009F448C0853B910509F447C0863B9105AF
:100B900009F446C0873B910509F445C0883B91059F
:100BA00009F444C0893B910509F443C08A3B91058F
:100BB00009F442C080E094E4089580E090E0089554
:100BC00081E890E4089583E890E4089582EE94E447
:100BD000089589EE94E408958AEE94E4089585EBEF
:100BE00094E4089586EB94E4089587EB94E40895E3
:100BF0008CEC94E408958DEC94E4089583E895E4F6
:100C000008958AE895E4089582E995E4089584E9D1
:100C100095E4089581E296E4089583E296E40895C8
:100C200084E296E4089585E296E4089586E296E4E7
:100C3000089587E296E408958AE296E40895089577
:100C400024E5829FC0011124FC0126E0729FE00D83
:100C5000F11D1124E60FF11DEE0FFF1FE052FF4FB3
:100C6000859194910895880F991FFC01E05AF040F6
:100C7000859194910895880F991FFC01E052FF4FD0
:100C800085919491089524E5829FC0011124FC016F
:100C900046E0749FE00DF11D1124E60FF11DEE0FEB
:100CA000FF1FE052FF4F859194919C013A952115C9
:100CB0004FE1340708F425C13F512115304120F49C
:100CC0009F700E943B0608959C01305321153041CE
:100CD00018F49927906C0895811520E5920769F41E
:100CE0000E94F5134FEF84E39CE041508040904018
:100CF000E1F700C000000C94FC1A813020E5920757
:100D000031F48091D00181608093D00108959C01DD
:100D100030552115304108F05CC0292F33272F7042
:100D2000332721303105E9F4AC0164E0440F551F4D
:100D30006A95E1F744275370BC016370772702C0BE
:100D4000220F331F6A95E2F73C68242B352B73E0A2
:100D5000880F991F7A95E1F780769927822B932B3C
:100D600008952230310529F4982F8827816F906AE1
:100D7000089523303105A1F4AC0133E0440F551F31
:100D80003A95E1F7407E57708370992721E030E073
:100D900002C0220F331F8A95E2F7C9019C6816C072
:100DA0002430310531F5AC0123E0440F551F2A955D
:100DB000E1F7407E57708370992721E030E002C050
:100DC000220F331F8A95E2F7C9019A68842B952B6D
:100DD00008959C0130572115304118F49F7090629E
:100DE00008959C0130582115304118F49F70906A85
:100DF0000895803E9105E0F4803C910558F58133DB
:100E0000910509F46FC048F48932910509F463C073
:100E10008A32910509F46DC072C089339105E9F0F9
:100E200082389105D1F08533910509F44DC067C032
:100E3000833E910581F138F4803E9105B9F0823E00
:100E40009105D9F05CC0863E910561F1873E910520
:100E5000A1F155C00E94330608952091E20120FDC2
:100E600002C021FF4CC080EE90E049C08091E201B9
:100E700080FFF9CF89E390E042C08091E20182FFD8
:100E80000EC08091E20184FF03C080E090E037C093
:100E900083EE90E034C08091E20182FFF2CF82EED7
:100EA00090E02DC08091E20183FF0BC08091E201B0
:100EB00084FDEBCF87EE90E022C08091E20183FFBA
:100EC000F5CF86EE90E01BC08091E20185FF07C060
:100ED00089E290E014C08091E20185FFF9CF85E3BB
:100EE00090E00DC08091E20186FF07C08AE290E0A9
:100EF00006C08091E20186FFF9CF81E390E00E9475
:100F00005F0508950895809166010895CF93DF935A
:100F100000D01F92CDB7DEB79C018091E8018430EC
:100F200019F593E099833B832A839093E9008FEF2F
:100F30009091E800815095FD06C095ED9A95F1F7E6
:100F400000008111F5CF8091E80085FF0DC040E0E1
:100F500050E063E070E0CE0101960E94F3098091B9
:100F6000E8008E778093E8000F900F900F90DF914C
:100F7000CF910895CF93DF9300D01F92CDB7DEB706
:100F80002091E801243021F522E029839B838A8384
:100F900083E08093E9008FEF9091E800815095FD08
:100FA00006C095ED9A95F1F700008111F5CF80917B
:100FB000E80085FF0DC040E050E063E070E0CE0146
:100FC00001960E94F3098091E8008E778093E800F3
:100FD0000F900F900F90DF91CF9108959C01809119
:100FE000E8018430F9F482E08093E9009FEF80917A
:100FF000E800915085FD06C085ED8A95F1F7000067
:101000009111F5CF8091E80085FF0CC040E050E0E1
:1010100065E070E0C9010E94F3098091E8008E77D5
:101020008093E8000895CF93DF93EC018091E8016D
:10103000843009F046C090910C019923D9F0909129
:101040000D019923B9F08093E9008FEF9091E800AA
:10105000815095FD06C095E19A95F1F70000811148
:10106000F5CF8091E80085FF2CC040E050E060E1C2
:1010700070E017C081E08093E9008FEF9091E80065
:10108000815095FD06C095ED9A95F1F7000081110C
:10109000F5CF8091E80085FF14C040E050E068E0A3
:1010A00070E0CE010E94F3098091E8008E77809372
:1010B000E80080E1FE01A6E5B1E001900D928A957D
:1010C000E1F7DF91CF9108958091E701811109C087
:1010D0000E94840B0E94E10B8091E2008460809367
:1010E000E20008951092E701089508950C943221CA
:1010F0000E94921A0E9438210E948C0E0C94820742
:1011000042E061EC81E00E94FD0A42E061EC82E095
:101110000E94FD0A42E061EC83E00E94FD0A42E188
:1011200061EC84E00C94FD0A8091EA01833009F4BB
:1011300055C030F4813071F0823009F48EC00895CA
:101140008A3009F47AC08B3009F460C0893009F024
:101150009CC020C08091E901813A09F096C080913D
:10116000E800877F8093E8008091ED019091EE0187
:10117000892B21F460E186E591E003C060E080E026
:1011800090E070E00E943E0A8091E8008B778093A7
:10119000E80008958091E901813209F076C08091DC
:1011A000ED019091EE01009719F0039709F06DC0E1
:1011B0008091E800877F8093E8008091E80082FDBD
:1011C00005C08091E8018111F8CF5FC08091F100E6
:1011D000809366018091E8008B7753C08091E9018C
:1011E000813A09F052C08091ED019091EE01892B76
:1011F00009F04BC08091E800877F8093E8008091E0
:10120000E80080FFFCCF80910C0136C08091E9019D
:101210008132D9F58091ED019091EE01892BA9F5EC
:101220008091E800877F8093E8000E94320B8091D4
:10123000EB0180930C010C94F5138091E90181324C
:1012400021F58091E800877F8093E8000E94320BAF
:101250008091EC018093670108958091E901813AC2
:10126000A1F48091E800877F8093E8008091E800F6
:1012700080FFFCCF809167018093F1008091E800AE
:101280008E778093E8000C94320B089584B7877FA3
:1012900084BF0FB6F894A895809160008861809310
:1012A0006000109260000FBE90E080E80FB6F894E6
:1012B00080936100909361000FBE0E94DB0E0E943C
:1012C000840B0E94E10B8091E20084608093E20035
:1012D00078940E946C0E0E94DD0E82E091E00E94E4
:1012E000870E0E9420218091E801853069F40E94D8
:1012F000541A8091E6018823B1F30E947E1A882354
:1013000091F30E94DD09EFCF0E94E30EECCF292F6D
:10131000332723303105C9F060F42130310581F0E5
:101320002230310509F041C08DE690E02CE033E039
:1013300040C021323105E1F02232310531F135C0B2
:1013400082E190E029E733E034C0992781309105AC
:1013500049F028F0029749F5E8EDF2E005C0E8E031
:10136000F3E002C0E0EFF2E0849190E09F0121C041
:101370006430D8F4E62FF0E0EE0FFF1FEE5DFE4F75
:101380002081318189E090E014C0643070F470E015
:10139000FB01EE0FFF1FE65EFE4F20813181FB0156
:1013A000EA5EFE4F808190E004C080E090E020E0A3
:1013B00030E0FA0131832083089580E189BD82E124
:1013C00089BD09B400FEFDCF8091D8008F7D809348
:1013D000D8008091E00082608093E0008091E0007E
:1013E00081FDFCCF0895CF92DF92EF92FF920F9391
:1013F0001F93CF93DF93EC018B016A010E94510B85
:10140000811133C0C114D10439F0F601808191817A
:10141000081B190BC80FD91FE12CF12C0115110560
:1014200019F18091E80085FD16C08091E8008E7763
:101430008093E800C114D10449F0F60180819181C4
:10144000E80EF91EF182E08285E00FC00E94510B88
:10145000882321F30AC089918093F100015011097A
:10146000FFEFEF1AFF0ADACF80E0DF91CF911F91F3
:101470000F91FF90EF90DF90CF9008952091EF01B2
:101480003091F0012617370748F06115710539F4DE
:101490002091E8002E772093E80001C0B901FC01FB
:1014A00020E06115710579F18091E8018823F1F15F
:1014B0008530F1F18091E80083FD3CC08091E80027
:1014C00082FD2EC08091E80080FFEBCF2091F300D9
:1014D0008091F20090E0922B6115710551F08830F7
:1014E000910538F421912093F10061507109019622
:1014F000F3CF21E0089709F020E08091E8008E7793
:101500008093E800CECF2111CFCF0AC08091E801AF
:10151000882361F0853061F08091E80083FD0AC086
:101520008091E80082FFF2CF80E0089582E0089584
:1015300083E0089581E008952091EF013091F0015A
:101540002617370748F06115710539F42091E80036
:101550002E772093E80001C0B901FC0120E061155D
:10156000710591F18091E801882309F440C085302C
:1015700009F43FC08091E80083FD3DC08091E80000
:1015800082FD2FC08091E80080FFE9CF2091F30019
:101590008091F20090E0922B6115710559F088302E
:1015A000910540F424912093F10031966150710926
:1015B0000196F2CF21E0089709F020E08091E80041
:1015C0008E778093E800CBCF2111CCCF0AC08091D9
:1015D000E801882361F0853061F08091E80083FDA7
:1015E0000AC08091E80082FFF2CF80E0089582E097
:1015F000089583E0089581E00895982F973068F565
:101600009093E900981739F07091EC002091ED006B
:101610005091F00003C0242F762F50E021FD02C02E
:101620009F5FECCF3091EB003E7F3093EB00309129
:10163000ED003D7F3093ED003091EB003160309351
:10164000EB007093EC002093ED005093F00020919C
:10165000EE0027FDE5CF80E008958F708093E900CC
:1016600081E008958091E90187FF11C08091E80031
:1016700082FD05C08091E8018111F8CF11C08091F1
:10168000E8008B770BC08091E801882349F08091B6
:10169000E80080FFF8CF8091E8008E778093E80023
:1016A00008952091E4003091E50095E64091EC002A
:1016B000842F817040FF23C08091E80080FD1DC011
:1016C0008091E801882399F0853099F08091EB00B2
:1016D00085FD11C04091E4005091E50024173507C5
:1016E00029F3915011F09A01E1CF84E0089582E04E
:1016F000089583E0089581E0089580E00895409181
:10170000E80042FFDDCF08950E94F20B0E94FA0B21
:10171000E0EEF0E0808181608083E8EDF0E08081A0
:101720008F77808319BCA7EDB0E08C918E7F8C936E
:1017300080818F7E80831092E70108950F931F931D
:10174000CF93DF930E94F20B0E94FA0BC8EDD0E01A
:1017500088818F77888388818068888388818F7D5E
:10176000888319BC1092E8011092E4011092E601FE
:101770001092E50100EE10E0F80180818B7F8083FC
:1017800088818160888342E060E080E00E94FD0AF9
:10179000E1EEF0E080818E7F8083E2EEF0E08081F8
:1017A00081608083808188608083F80180818E7F62
:1017B0008083888180618883DF91CF911F910F9111
:1017C0000895E8EDF0E080818F7E8083E7EDF0E022
:1017D00080818160808384E082BF81E08093E70123
:1017E0000C949E0BE8EDF0E080818E7F8083109258
:1017F000E20008951092DA001092E10008951F921D
:101800000F920FB60F9211242F933F934F935F9334
:101810006F937F938F939F93AF93BF93EF93FF93B8
:101820008091E10082FF0BC08091E20082FF07C03F
:101830008091E1008B7F8093E1000E946B0E80918C
:10184000DA0080FF1FC08091D80080FF1BC080910C
:10185000DA008E7F8093DA008091D90080FF0DC07E
:1018600080E189BD82E189BD09B400FEFDCF81E040
:101870008093E8010E94640805C019BC1092E80139
:101880000E9472088091E10080FF19C08091E200FF
:1018900080FF15C08091E2008E7F8093E2008091EE
:1018A000E20080618093E2008091D80080628093A2
:1018B000D80019BC85E08093E8010E9476088091E9
:1018C000E10084FF30C08091E20084FF2CC080E101
:1018D00089BD82E189BD09B400FEFDCF8091D800A9
:1018E0008F7D8093D8008091E1008F7E8093E1000E
:1018F0008091E2008F7E8093E2008091E20081601F
:101900008093E2008091E401882311F084E007C015
:101910008091E30087FD02C081E001C083E08093F5
:10192000E8010E9478088091E10083FF29C080913E
:10193000E20083FF25C08091E100877F8093E10072
:1019400082E08093E8011092E4018091E1008E7FB3
:101950008093E1008091E2008E7F8093E20080918D
:10196000E20080618093E20042E060E080E00E945B
:10197000FD0A8091F00088608093F0000E94750855
:10198000FF91EF91BF91AF919F918F917F916F9157
:101990005F914F913F912F910F900FBE0F901F902D
:1019A00018951F920F920FB60F9211242F933F9309
:1019B0004F935F936F937F938F939F93AF93BF9357
:1019C000CF93DF93EF93FF93C091E900CF708091A5
:1019D000EC00D82FD17080FDD0E81092E900809102
:1019E000F000877F8093F00078940E94150D10928C
:1019F000E9008091F00088608093F000CD2BCF70DB
:101A0000C093E900FF91EF91DF91CF91BF91AF912A
:101A10009F918F917F916F915F914F913F912F9106
:101A20000F900FBE0F901F9018951F93CF93DF93C9
:101A3000CDB7DEB7AA970FB6F894DEBF0FBECDBF05
:101A4000E9EEF1E08091F100819321E0E13FF207BE
:101A5000C9F70E9494088091E80083FF24C1809117
:101A6000E9019091EA01492F50E04A30510508F010
:101A70001AC1FA01EA5AFF4F0C94C922803881F04A
:101A8000823809F010C18091ED018F708093E900D8
:101A90008091EB0085FB882780F91092E90006C051
:101AA0008091E5019091E601911182609091E800AA
:101AB000977F9093E8008093F1001092F100C8C0E6
:101AC000282F2D7F09F0EFC0882319F0823061F0B4
:101AD000EAC08091EB01813009F0E5C0933009F054
:101AE00080E08093E6012BC08091EB01811127C03B
:101AF0008091ED018F7009F4D6C08093E9002091A8
:101B0000EB0020FF1CC0933021F48091EB00806239
:101B100014C09091EB0090619093EB0021E030E0D5
:101B2000A90102C0440F551F8A95E2F74093EA00CD
:101B30001092EA008091EB0088608093EB00109295
:101B4000E9008091E800877F86C08111ACC01091C8
:101B5000EB011F778091E3008078812B8093E30075
:101B60008091E800877F8093E8000E94320B80918B
:101B7000E80080FFFCCF8091E30080688093E30061
:101B8000111102C082E001C083E08093E8018BC0A4
:101B90008058823008F087C08091EB019091EC0171
:101BA0008C3D53E0950779F583E08A838AE2898347
:101BB0004FB7F894DE01139620E03EE051E2E32FA8
:101BC000F0E050935700E49120FF03C0E295EF70DE
:101BD0003F5FEF708E2F90E0EA3010F0C79601C0A3
:101BE000C0968D939D932F5F243149F74FBF80910D
:101BF000E800877F8093E8006AE270E0CE010196FA
:101C00000E943E0A14C0AE014F5F5F4F6091ED012C
:101C10000E948709BC01892B09F445C09091E80016
:101C2000977F9093E80089819A810E949C0A809115
:101C3000E8008B778093E80036C08038A1F580916A
:101C4000E800877F8093E8008091E4018093F100B1
:101C50008091E8008E778093E8000E94320B23C0C9
:101C6000811121C08091EB019091EC01992702979D
:101C7000D4F48091E800877F8093E8008091EB01A5
:101C80008093E4010E94320B8091E401811106C02F
:101C90008091E30087FD02C081E001C084E0809371
:101CA000E8010E9480088091E80083FF0AC08091CB
:101CB000E800877F8093E8008091EB00806280934A
:101CC000EB00AA960FB6F894DEBF0FBECDBFDF9132
:101CD000CF911F9108950895CF938091E8018823B3
:101CE000A1F0C091E900CF709091EC00892F817034
:101CF00090FD80E8C82B1092E9008091E80083FDF8
:101D00000E94150DCF70C093E900CF910895909374
:101D10006D0180936C010895E0916C01F0916D016B
:101D2000309721F00190F081E02D099480E0089532
:101D3000E0916C01F0916D01309721F00280F38108
:101D4000E02D09940895E0916C01F0916D013097B8
:101D500021F00480F581E02D0994089520916A0115
:101D600030916B012817390771F090936B018093C4
:101D70006A01E0916C01F0916D01309721F00680CD
:101D8000F781E02D0994089520916801309169014F
:101D90002817390771F09093690180936801E091E9
:101DA0006C01F0916D01309721F00084F185E02DF8
:101DB0000994089508950C94DA0E0E94981A0E94CE
:101DC0004A040C945E1BCF92DF92EF92FF920F9326
:101DD0001F93CF93DF93CDB7DEB72B970FB6F89451
:101DE000DEBF0FBECDBF0E9462048FE6C82E81E029
:101DF000D82E00E010E0E02E802F0E945805F6015A
:101E000041916F01F82EF426B1F40F5F1F4F0E3091
:101E1000110589F78FEF89838A831B820E94A11A9B
:101E20008160782F9D838C8349815A816B818D815C
:101E30000E94860F40C09091D00191FF04C08B8713
:101E40000E945E058B8520E030E04F2D50E0922F00
:101E5000BA01022E02C0759567950A94E2F760FFF9
:101E600024C02E83EF8221E030E0690102C0CC0C57
:101E7000DD1C9A95E2F790E08C219D21892B09F4D5
:101E800020E028870E94A11A8160782F9A8789878D
:101E90004E815F8168858A850E94860FF801E1592D
:101EA000FE4F8081C826C08206C02F5F3F4F26307C
:101EB000310569F6AACF0E94451E0E948C0E9091B2
:101EC0006E018917A1F00E948C0E80936E012B96F3
:101ED0000FB6F894DEBF0FBECDBFDF91CF911F913B
:101EE0000F91FF90EF90DF90CF900C9482072B968C
:101EF0000FB6F894DEBF0FBECDBFDF91CF911F911B
:101F00000F91FF90EF90DF90CF900895CF93DF93E4
:101F1000CDB7DEB72B970FB6F894DEBF0FBECDBF9F
:101F20004F83588769877A878B87DE01119686E011
:101F3000FD0111928A95E9F785E0FE01379601903F
:101F40000D928A95E1F749815A816B817C818D815F
:101F50009E810E9489162B960FB6F894DEBF0FBEA5
:101F6000CDBFDF91CF910895CF93C82F882309F477
:101F7000C1C0823859F40E948C0E81FDBBC089E338
:101F80000E9426190E94DE1989E30CC0833879F477
:101F90000E948C0E80FDAEC083E50E9426190E942F
:101FA000DE1983E50E946519CF910C94DE198438FF
:101FB00059F40E948C0E82FD9DC087E40E94261970
:101FC0000E94DE1987E4EECF8CEF8C0F813A48F443
:101FD0008C2F0E94852081118DC08C2F0E94261984
:101FE000E3CF80E28C0F883048F4C77081E001C0F5
:101FF000880FCA95EAF70E94A719D6CF8BE58C0FF8
:10200000833078F4C53A29F0C63A31F083E890E09D
:1020100005C081E890E002C082E890E0CF910C9486
:10202000AE0E88E58C0F833108F064C0C83A39F1F0
:10203000C93A41F1CA3A49F1CB3A51F1CC3A59F196
:10204000CD3A61F1C03B69F1CE3A71F1CF3A79F105
:10205000C13B81F1C23B89F1C33B91F1C43B99F192
:10206000C53BA1F1C63BA9F1C73BB1F1C83BB9F1F2
:10207000C93BC1F1CA3BC9F180E090E038C082EEB3
:1020800090E035C089EE90E032C08AEE90E02FC03B
:1020900085EB90E02CC086EB90E029C087EB90E0C8
:1020A00026C08CEC90E023C08DEC90E020C083E84B
:1020B00091E01DC08AE891E01AC082E991E017C062
:1020C00084E991E014C081E292E011C083E292E0E1
:1020D0000EC084E292E00BC085E292E008C086E286
:1020E00092E005C087E292E002C08AE292E0CF91DE
:1020F0000C94C40ECF910895882309F44BC0823804
:1021000059F40E948C0E81FF45C089E30E94261974
:102110000E94DE1989E30CC0833871F40E948C0E92
:1021200080FF38C083E50E9426190E94DE1983E5EE
:102130000E9465190C94DE19843859F40E948C0EA3
:1021400082FF28C087E40E9426190E94DE1987E4D6
:10215000EFCF9CEF980F913A58F390E2980F983098
:1021600050F4877091E001C0990F8A95EAF7892FA2
:102170000E94AD19DFCF9BE5980F933020F480E0EB
:1021800090E00C94AE0E885A833120F480E090E009
:102190000C94C40E0895882321F00E94A7190C9472
:1021A000DE190895882321F00E94AD190C94DE19E0
:1021B0000895BF92CF92DF92EF92FF920F931F93F9
:1021C000CF93DF9300D000D000D0CDB7DEB77C0135
:1021D00085E0F701DE01119601900D928A95E1F7F5
:1021E000F70183819481892B09F4DDC2908181817B
:1021F0008F3F19F49F3F09F4D6C2F7010281258170
:1022000022952F7099838A8389819A812E830E94D7
:10221000E518182FB92E0E94E4180E94AB17EB2D79
:10222000E295EF704E2F50E0FA01E05AFF4F2E81F9
:102230000C94C9228B2D807F9B2D9F70F92E8823B3
:1022400019F0F29480EFF822002349F0FF2009F4FE
:1022500057C28F2D0E94B7190E94DE1951C2812FDB
:102260000E947C10FF2009F49EC28F2D0E94BD1990
:1022700026960FB6F894DEBF0FBECDBFDF91CF918B
:102280001F910F91FF90EF90DF90CF90BF900C9433
:10229000DE193B2D307F8B2D8F70303211F08295FF
:1022A000807F112319F0113021F12CC00023B9F0E7
:1022B000222309F490C1213009F08DC126960FB672
:1022C000F894DEBF0FBECDBFDF91CF911F910F916C
:1022D000FF90EF90DF90CF90BF900C94C71922230E
:1022E00019F0213009F45FC28E830E94CA198E81D1
:1022F00086C1002321F0223008F055C26CC12111A3
:1023000052C27DC1002321F0222309F464C1F8C127
:10231000222309F474C109C28B2D8695869583709A
:1023200019F08130D1F03FC2002321F0812F9B2D85
:10233000937002C080E090E026960FB6F894DEBF5E
:102340000FBECDBFDF91CF911F910F91FF90EF9006
:10235000DF90CF90BF900C94AE0E002321F0812F20
:102360009B2D937002C080E090E026960FB6F89403
:10237000DEBF0FBECDBFDF91CF911F910F91FF90B8
:10238000EF90DF90CF90BF900C94C40E812F00236C
:1023900019F00E944D1D02C00E94B51D26960FB671
:1023A000F894DEBF0FBECDBFDF91CF911F910F918B
:1023B000FF90EF90DF90CF90BF900C943A1E8B2D42
:1023C000837009F075C00111EEC1812F8295869549
:1023D0008770880F880F912F9F70C92ED12CE12C08
:1023E000F12C082E04C0CC0CDD1CEE1CFF1C0A9442
:1023F000D2F714FF12C00FE010E020E030E004C07C
:10240000000F111F221F331F8A95D2F7C901B8018F
:10241000609570958095909503C060E070E0CB0169
:102420004B2D4695469543704230C1F060F56C29BE
:102430007D298E299F29413051F126960FB6F894B7
:10244000DEBF0FBECDBFDF91CF911F910F91FF90E7
:10245000EF90DF90CF90BF900C94D2176C297D291C
:102460008E299F2926960FB6F894DEBF0FBECDBFEA
:10247000DF91CF911F910F91FF90EF90DF90CF9060
:10248000BF900C94EE170E94D217C701B601269692
:102490000FB6F894DEBF0FBECDBFDF91CF911F9175
:1024A0000F91FF90EF90DF90CF90BF900C94B617F4
:1024B000002319F08B2D817001C08695882309F4C3
:1024C00072C1812F829586958770880F880F912F12
:1024D0009F70C92ED12CE12CF12C082E04C0CC0CFD
:1024E000DD1CEE1CFF1C0A94D2F714FF12C00FE093
:1024F00010E020E030E004C0000F111F221F331F46
:102500008A95D2F7C901B80160957095809590952C
:1025100003C060E070E0CB014B2D469546954370BB
:102520004230C1F060F56C297D298E299F29413008
:1025300051F126960FB6F894DEBF0FBECDBFDF91E6
:10254000CF911F910F91FF90EF90DF90CF90BF90B0
:102550000C94AC186C297D298E299F2926960FB6DC
:10256000F894DEBF0FBECDBFDF91CF911F910F91C9
:10257000FF90EF90DF90CF90BF900C94C8180E940E
:10258000AC18C701B60126960FB6F894DEBF0FBE91
:10259000CDBFDF91CF911F910F91FF90EF90DF9012
:1025A000CF90BF900C949018103FD1F118F4103ECA
:1025B00050F4A1C0123F09F463C008F44CC0133FAB
:1025C00009F473C098C01F708B2D8F710023A1F088
:1025D0000E942918812F26960FB6F894DEBF0FBEF1
:1025E000CDBFDF91CF911F910F91FF90EF90DF90C2
:1025F000CF90BF900C94CB100E944A18812F269642
:102600000FB6F894DEBF0FBECDBFDF91CF911F9103
:102610000F91FF90EF90DF90CF90BF900C94D2106D
:102620000023A9F02111BFC08B2D8F7126960FB604
:10263000F894DEBF0FBECDBFDF91CF911F910F91F8
:10264000FF90EF90DF90CF90BF900C946F182230E6
:1026500008F0A9C0E9CF0023A9F08B2D8F71269631
:102660000FB6F894DEBF0FBECDBFDF91CF911F91A3
:102670000F91FF90EF90DF90CF90BF900C942918AE
:10268000002359F38B2D8F7126960FB6F894DEBF79
:102690000FBECDBFDF91CF911F910F91FF90EF90B3
:1026A000DF90CF90BF900C944A18002399F08B2DA7
:1026B0008F7126960FB6F894DEBF0FBECDBFDF91A7
:1026C000CF911F910F91FF90EF90DF90CF90BF902F
:1026D0000C94141826960FB6F894DEBF0FBECDBF2B
:1026E000DF91CF911F910F91FF90EF90DF90CF90EE
:1026F000BF900C940A180023A9F0222309F4ADCF4F
:10270000812F26960FB6F894DEBF0FBECDBFDF91A6
:10271000CF911F910F91FF90EF90DF90CF90BF90DE
:102720000C94B40F222309F4ADCF812F26960FB657
:10273000F894DEBF0FBECDBFDF91CF911F910F91F7
:10274000FF90EF90DF90CF90BF900C947C104B2DBA
:102750004F70612FC7010E94AC0226960FB6F89405
:10276000DEBF0FBECDBFDF91CF911F910F91FF90C4
:10277000EF90DF90CF90BF900C942E174B2D4F70A1
:10278000612FC70126960FB6F894DEBF0FBECDBFEE
:10279000DF91CF911F910F91FF90EF90DF90CF903D
:1027A000BF900C941F0626960FB6F894DEBF0FBE9E
:1027B000CDBFDF91CF911F910F91FF90EF90DF90F0
:1027C000CF90BF9008950E94C4190E9499190E9449
:1027D000DE190E94EA1E0E943A1E80E090E00E94EC
:1027E000AE0E80E090E00C94C40E0E94B4190C94DC
:1027F000E3130E94E518292F22952F702C3030F416
:102800002A3048F42250223078F405C02C3041F0B0
:102810002F3031F009C0803E48F0803F29F406C0D7
:1028200093FB882780F9089580E0089581E008955A
:10283000CF93DF9300D000D01F92CDB7DEB70F90BB
:102840000F900F900F900F90DF91CF910895CF933D
:10285000DF9300D000D000D0CDB7DEB726960FB6FC
:10286000F894DEBF0FBECDBFDF91CF9108951F93C7
:10287000CF93DF93C0917D0116E080917E01C81750
:1028800099F0D0E01C9FF0011D9FF00D1124E1583C
:10289000FE4F4081518162817381848195810E94C4
:1028A00027142196C770E9CFDF91CF911F9108952A
:1028B0004091AF015091B0016091B1017091B201AE
:1028C0008091B3019091B4010C9427148091B401CC
:1028D00082958F7009F054C08091B101882309F46A
:1028E0004FC080917D01A0917E014091B201509135
:1028F000B3016091AF017091B001B6E08A1709F49D
:102900003FC090E041155105C1F17F3F11F46F3F89
:10291000A1F1B89FF001B99FF00D1124E158FE4FCD
:10292000218127132AC02081261327C0228121114B
:1029300024C0238134812417350710F42150310934
:10294000241B350B283C3105C0F42091B4012F70B5
:1029500020612093B40126E0289FF001299FF00D0B
:102960001124EC57FE4F80818F70806180838FEA45
:1029700091E00E94D9100C94371401968770BECF55
:102980000895CF92DF92EF92FF920F931F93CF9310
:10299000DF93CDB7DEB762970FB6F894DEBF0FBEF8
:1029A000CDBF8C0185E0F801DE011D9601900D92EE
:1029B0008A95E1F7D8014C9111965C911197129686
:1029C0006C918091B2019091B301009709F475C1A7
:1029D0003091AF017091B0017F3F19F43F3F09F48E
:1029E0006CC1F801C380D480E090B101EE2009F4FD
:1029F000BEC02091B401C816D90628F0D601A81B84
:102A0000B90BCD0104C0809590958C0D9D1DFF24C0
:102A1000F394883C910578F0F12C207F09F0C4C034
:102A20007C2DD98AC88A89890E9418148FEA91E07E
:102A30000E94D910AFC0822F807F09F045C0571384
:102A400013C0431311C061110FC02F702061209378
:102A5000B4010E9458148FEA91E00E94D91080912D
:102A6000B401F80185832EC0CD2819F15F3F11F420
:102A70004F3FF9F0F62E61111CC080917D0120912D
:102A80007E0136E0821709F45BC090E0389FF001C8
:102A9000399FF00D1124E158FE4F7181571306C084
:102AA0007081471303C07281711103C00196877052
:102AB000E9CFF62E662309F41CC18091B401816030
:102AC0008093B401F12C15C1571309C0431307C0FB
:102AD000611105C08091B401F8018583C8C04D879C
:102AE0005E878D859E856A8B0E94F9136A8988238B
:102AF000D1F16623C1F12091B401822F82958F70AC
:102B000090E0029774F08091AF019091B0019887A6
:102B10008F831986DB86CA862C87CE0107960E9492
:102B2000D91086E0F801AFEAB1E001900D928A95E4
:102B3000E1F70E9466140E945814FF24F394D9C050
:102B40004D875E878D859E850E94E518292F2295E9
:102B50002F70223008F0C1C09F7009F0BBC0805EAA
:102B6000883008F4C6C0C8010E94D910E6CFC81644
:102B7000D90608F453C0F601E81BF90BCF01883CD5
:102B8000910508F450C0F12C7C2DD98AC88A898916
:102B90000E941814EFEAF1E086E0DF011D928A95A9
:102BA000E9F70E945814A5C0571314C0431312C06C
:102BB000611110C08091B401F8018583C8010E94A1
:102BC000D91086E0EFEAF1E0DF011D928A95E9F77E
:102BD000FE2C8FC04D875E878D859E856A8B0E94F7
:102BE000F9136A89882309F4BECF662309F4BBCFA1
:102BF0002091B401822F82958F7090E002970CF49F
:102C000090CF8091AF019091B0019A8389831B820C
:102C1000DD82CC822E83CE01019681CF8095909566
:102C20008C0D9D1DACCFF62E662309F49CCF571357
:102C300033C0431331C02091B40120FD24C0822F42
:102C400082958F70482F50E041155105E1F0D80171
:102C500015962C9315974F30510549F08F5F982F9B
:102C60009295907F822F8F70892B15968C93C80137
:102C70000E94D91086E0F801AFEAB1E001900D9210
:102C80008A95E1F78ECF86E0F801AFEAB1E00190D6
:102C90000D928A95E1F72DC04D875E878D859E85C3
:102CA0000E94F91381113DCF8091B401816080931E
:102CB000B401C8010E94D9101CC0662309F453CF87
:102CC0004D875E878D859E850E94F913882309F4C0
:102CD0004ACF27CF811143CF0CC0243008F043CF17
:102CE0009F7009F43CCFD80115969C91907F09F014
:102CF00036CF8F2D62960FB6F894DEBF0FBECDBFD4
:102D0000DF91CF911F910F91FF90EF90DF90CF90C7
:102D100008951F93CF93DF93CDB7DEB72C970FB6EF
:102D2000F894DEBF0FBECDBF4F83588769877A877F
:102D30008B879C87CE0107960E94C114882371F06F
:102D40008A859B85892B09F441C088858F3F09F0CE
:102D500065C08F818F3F09F061C038C086E0FE01F9
:102D60003796DE01119601900D928A95E1F76A85FA
:102D70007B856115710551F1FF81E885EF3F11F405
:102D8000FF3F21F120917E0130E0C901019687705B
:102D9000992740917D0150E08417950709F447C0B9
:102DA000F983EA837D836C8396E0929FD001939FA1
:102DB000B00D1124A158BE4FFE01319601900D9225
:102DC0009A95E1F780937E010E94371416E0809176
:102DD0007D0190917E018917B9F1189FC0011124DE
:102DE00081589E4F0E94C114882371F1E0917D01AA
:102DF0001E9FF0011124E158FE4F408151816281F4
:102E00007381848195810E94271480917D0190E0D7
:102E100001968770992780937D01D9CF4F8158857E
:102E200069857A858B859C850E942714CFCF0E9467
:102E3000F51310927E0110927D01EFEAF1E086E039
:102E4000DF011D928A95E9F72C960FB6F894DEBF44
:102E50000FBECDBFDF91CF911F910895EF92FF92EA
:102E60000F931F93CF93DF938C01892B09F46CC0D0
:102E7000F12CEE24E394E8012196F8018491843743
:102E800040F4843008F051C0813081F0823019F173
:102E90005BC0853709F444C0A8F19CE7980F9037D0
:102EA00008F052C08F770E947C1041C00E5F1F4F08
:102EB000FE01849190E2980F983050F48770FE2DB7
:102EC00001C0FF0F8A95EAF78F2F0E94B71914C02F
:102ED0000E94B40F2DC00E5F1F4FFE01849190E23F
:102EE000980F983060F48770FE2D01C0FF0F8A950F
:102EF000EAF78F2F0E94BD190E94DE1919C00E94A7
:102F00007C1016C00E5F1F4FFE01C491CC2381F0D0
:102F10008FE99FE00197F1F700C00000C150F6CFA4
:102F20000E5F1F4FFE01F49003C00E94B40F8E018C
:102F30008F2D882309F49FCFEFE9FFE03197F1F758
:102F400000C000008150F5CFDF91CF911F910F910C
:102F5000FF90EF90089508956093B9017093BA01BE
:102F60008093BB019093BC010C94E3130F931F93C8
:102F70000091B9011091BA012091BB013091BC01BF
:102F8000DC01CB01802B912BA22BB32B8093B901B9
:102F90009093BA01A093BB01B093BC011F910F9114
:102FA0000C94E3130F931F930091B9011091BA0190
:102FB0002091BB013091BC01DC01CB018023912326
:102FC000A223B3238093B9019093BA01A093BB01CC
:102FD000B093BC011F910F910C94E3130F931F93B7
:102FE0000091B9011091BA012091BB013091BC014F
:102FF000DC01CB0180279127A227B3278093B90159
:103000009093BA01A093BB01B093BC011F910F91A3
:103010000C94E3131092B5011092B6011092B7010F
:103020001092B8010C94E31341E050E060E070E0CE
:1030300004C0440F551F661F771F8A95D2F740932F
:10304000B5015093B6016093B7017093B8010C9429
:10305000E31341E050E060E070E004C0440F551F0E
:10306000661F771F8A95D2F78091B5019091B601BE
:10307000A091B701B091B801482B592B6A2B7B2B3B
:103080004093B5015093B6016093B7017093B801B6
:103090000C94E31341E050E060E070E004C0440FA2
:1030A000551F661F771F8A95D2F7409550956095FA
:1030B00070958091B5019091B601A091B701B09142
:1030C000B801482359236A237B234093B5015093C9
:1030D000B6016093B7017093B8010C94E31341E01B
:1030E00050E060E070E004C0440F551F661F771F7A
:1030F0008A95D2F78091B5019091B601A091B70160
:10310000B091B801482759276A277B274093B5011A
:103110005093B6016093B7017093B8010C94E31318
:103120000F931F930091B5011091B6012091B70143
:103130003091B801DC01CB01802B912BA22BB32B5A
:103140008093B5019093B601A093B701B093B801F5
:103150001F910F910C94E3130F931F930091B501EE
:103160001091B6012091B7013091B801DC01CB017B
:1031700080239123A223B3238093B5019093B601BA
:10318000A093B701B093B8011F910F910C94E31372
:103190000F931F930091B5011091B6012091B701D3
:1031A0003091B801DC01CB0180279127A227B327FA
:1031B0008093B5019093B601A093B701B093B80185
:1031C0001F910F910C94E3130895CF92DF92EF9229
:1031D000FF920F931F93CF93DF938C01C090B501A3
:1031E000D090B601E090B701F090B8018091B9019C
:1031F0009091BA01A091BB01B091BC01C82AD92A13
:10320000EA2AFB2ACFE1D0E0D701C6010C2E04C088
:10321000B695A795979587950A94D2F780FF07C032
:10322000B8018C2F0E9443068130910531F421971B
:1032300058F7B80180E00E944306DF91CF911F91BB
:103240000F91FF90EF90DF90CF90089590910C0137
:103250009923F1F090910D019923D1F0982F969533
:10326000969596959F3080F5E0910E01F0910F01B3
:10327000E90FF11D877021E030E0A90102C0440F81
:10328000551F8A95E2F7CA019181892B81830895A0
:1032900020910E0130910F01F90132969FEF40E02D
:1032A0005191851789F09F3F19F4511101C0942F56
:1032B0004F5F4E30A9F79F3F39F0F901E90FF11D3B
:1032C00097FDFA9582830895089590910C019923B2
:1032D000F9F090910D019923D9F0982F9695969534
:1032E00096959F3028F5E0910E01F0910F01E90FBE
:1032F000F11D877021E030E0A90102C0440F551F85
:103300008A95E2F7CA018095918189238183089586
:1033100020910E0130910F01F9013296205F3F4F4D
:103320009081891301C010823196E217F307C1F72B
:10333000089581E090E0E0910E01F0910F01E80F17
:10334000F91F1082019680319105A9F70895909197
:10335000CF01892B8093CF01089580959091CF0163
:1033600089238093CF0108951092CF010895909101
:10337000CE01892B8093CE01089580959091CE0146
:1033800089238093CE0108951092CE0108958093F1
:10339000BD0108951092BD01089580910E01909194
:1033A0000F01FC0131969C01205F3F4F80E091911D
:1033B00091118F5FE217F307D1F70895E0910E01A5
:1033C000F0910F018091CF018083E0910E01F09187
:1033D0000F0190818091CE01892B80838091BD0166
:1033E000882361F0E0910E01F0910F019081892B0B
:1033F00080830E94CD1981111092BD0180910E0130
:1034000090910F010C94980ECF92DF92EF92FF9261
:103410006C01EE24FF24C114D104E104F10421F075
:10342000C701B60120E101C020E0C72ED82EE92E49
:10343000FF24C114D104E104F10419F0285FC7018D
:10344000B6016B017C0154E0F694E794D794C794DD
:103450005A95D1F7C114D104E104F10419F02C5F9D
:10346000C701B6016B017C0142E0F694E794D79462
:10347000C7944A95D1F7C114D104E104F10419F0BD
:103480002E5FC701B601DC01CB01B695A7959795D4
:103490008795892B8A2B8B2B09F02F5F822FFF902A
:1034A000EF90DF90CF9008958091E801843011F182
:1034B00020E488E190E00FB6F894A895809360002E
:1034C0000FBE2093600083B7817F846083BF83B782
:1034D000816083BF7894889583B78E7F83BF0FB652
:1034E000F894A895809160008861809360001092A4
:1034F00060000FBE089508950C947B1ACF930E942C
:103500007C1A0E9462040E947B1AC0E08C2F0E94E9
:103510005805811104C0CF5FCE30C1F701C081E0F2
:10352000CF9108950E94F5130E948C0E0C9482078F
:1035300082E084BD93E095BD9AEF97BD80936E00C5
:1035400008952FB7F8948091D1019091D201A09164
:10355000D301B091D4012FBF0895CF92DF92EF92A3
:10356000FF920F931F932FB7F8944091D101509180
:10357000D2016091D3017091D4012FBF6A017B0108
:10358000EE24FF248C0120E030E0C016D106E206D4
:10359000F30610F4415051099A01281B390BC90157
:1035A0001F910F91FF90EF90DF90CF9008951F92A1
:1035B0000F920FB60F9211248F939F93AF93BF93E7
:1035C0008091D1019091D201A091D301B091D40109
:1035D0000196A11DB11D8093D1019093D201A093BA
:1035E000D301B093D401BF91AF919F918F910F9070
:1035F0000FBE0F901F9018950E94840BF8942FEF28
:1036000087EA91E6215080409040E1F700C0000039
:1036100087E090EBDC018093F1019093F201A0939D
:10362000F301B093F4019CE088E10FB6F894A895FB
:10363000809360000FBE90936000FFCFEF92FF92E7
:103640000F931F93CF93DF93D82FC0E08C2F0E944E
:10365000580500E010E0E82EF12CC701002E02C052
:10366000959587950A94E2F780FD06C00F5F1F4F7E
:103670000630110591F709C0602F7C2F80E00E9471
:1036800020068D13F3CF81E004C0CF5FCE30F1F67A
:1036900080E0DF91CF911F910F91FF90EF900895FF
:1036A000CF93C82F8CE20E941E1B882321F08C2F01
:1036B000CF910C941E1B80E0CF910895CF930E9470
:1036C000A51C811102C00E948B1CC5E6C15049F0A7
:1036D0000E9462048FE39CE90197F1F700C00000AB
:1036E000F5CF89E20E94501B811113C18AE20E942A
:1036F000501B81110E948B1C85E00E94501B811180
:103700000E94FC1A0E94B01C8093D00187E00E94A6
:10371000501B8823A9F18BE10E94501B882351F094
:103720008091D00181FB222720F991E0922790FB24
:1037300081F90EC08EE00E94501B882361F08091B9
:10374000D00182FB222720F991E0922790FB82F999
:103750008093D00115C080E10E94501B9091D00150
:10376000882341F093FB222720F981E0822780FB08
:1037700093F904C0892F809580FB90F99093D00134
:103780008091D0010E94B41C0E94C21C8093E2016F
:1037900080EE0E94501B882341F08091E201982F17
:1037A000909590FB80F98093E20189E30E94501B81
:1037B000882359F08091E20181FB222720F991E0D2
:1037C000922790FB81F98093E20182EE0E94501BC8
:1037D000882359F08091E20182FB222720F991E0B1
:1037E000922790FB82F98093E20186EE0E94501BA3
:1037F000882359F08091E20183FB222720F991E090
:10380000922790FB83F98093E20183EE0E94501B84
:10381000882359F08091E20184FB222720F991E06E
:10382000922790FB84F98093E20185E30E94501B6C
:10383000882359F08091E20185FB222720F991E04D
:10384000922790FB85F98093E20181E30E94501B4F
:10385000882359F08091E20186FB222720F991E02C
:10386000922790FB86F98093E20181E10E94501B30
:10387000882359F08091E20187FB222720F991E00B
:10388000922790FB87F98093E2018091E2010E94E8
:10389000C61C8091E20187FB882780F980930D0187
:1038A00087E20E94501BC82F8EE10E94501B81119D
:1038B000C2608FE10E94501B8111C46080E20E94AF
:1038C000501B8111C86081E20E94501B8111C061B0
:1038D00082E20E94501B8111C06283E20E94501B51
:1038E0008111C06484E20E94501B882311F0C068DB
:1038F00002C0CC2329F08C2F0E94BD1C6C2F03C06A
:103900000E94B91C682F70E080E090E0CF910C9489
:10391000AC17CF9108956DEE7EEF80E090E00E94AD
:10392000FF2260E082E090E00E94F12260E083E00C
:1039300090E00E94F12260E084E090E00E94F12299
:1039400060E085E090E00C94F12280E090E00E943D
:10395000EB2221E08D3E9E4F09F020E0822F08955A
:1039600082E090E00C94E322682F82E090E00C94D7
:10397000F12283E090E00C94E322682F83E090E052
:103980000C94F12284E090E00C94E322682F84E010
:1039900090E00C94F1228091D70180FF0BC06091E0
:1039A000130185E0689FB0011124759567957595A1
:1039B00067952BC081FF09C06091130185E0689F66
:1039C000B00111247595679520C082FF07C06091F2
:1039D000130185E0689FB001112417C09091D801B0
:1039E0009923D1F060911201961788F72091130165
:1039F00085E0289F90011124929FA001939F500D74
:103A0000112470E0CA010E94B5226038710540F4AB
:103A10006115710519F406C065E070E0862F089500
:103A20008FE7089581E008958091D70180FF08C055
:103A30006091110170E0759567957595679521C046
:103A400081FF06C06091110170E07595679519C0FE
:103A500082FF04C06091110170E010C09091D80104
:103A6000992399F0609110019617A0F780911101A8
:103A7000899FC001112470E00E94B5226038710551
:103A800040F46115710519F406C061E070E0862FFD
:103A900008958FE7089581E00895803F21F40E9402
:103AA000CB1C819504C0813F29F40E94CB1C8093DC
:103AB000DB010895823F21F40E94CB1C819504C054
:103AC000833F29F40E94CB1C8093DA010895893F3B
:103AD00019F40E94141D05C08A3F31F40E94141D80
:103AE00081958093DC0108958B3F21F40E94141D81
:103AF000819504C08C3F29F40E94141D8093DD0140
:103B00000895843F21F48091D901816017C0853FD9
:103B100021F48091D901826011C0863F21F4809107
:103B2000D90184600BC0873F21F48091D90188605E
:103B300005C0883F31F48091D90180618093D9011B
:103B400008958D3F21F48091D70181600BC08E3F95
:103B500021F48091D701826005C08F3F29F48091C4
:103B6000D70184608093D7010895803F39F4809114
:103B7000DB0187FF6CC01092DB0169C0813F29F433
:103B80008091DB011816BCF362C09091DA01823F8C
:103B900029F497FF5CC01092DA0159C0833F19F4F1
:103BA0001916CCF354C0893F41F48091DC011816FA
:103BB0000CF04DC01092DC014AC08A3F29F480917C
:103BC000DC0187FF44C0F6CF8B3F39F48091DD01E3
:103BD00087FF3DC01092DD013AC08C3F29F48091EF
:103BE000DD011816BCF333C0843F21F48091D90164
:103BF0008E7F17C0853F21F48091D9018D7F11C040
:103C0000863F21F48091D9018B7F0BC0873F21F43F
:103C10008091D901877F05C0883F31F48091D90117
:103C20008F7E8093D90113C08D3F21F48091D701FD
:103C30008E7F0BC08E3F21F48091D7018D7F05C010
:103C40008F3F29F48091D7018B7F8093D70180919A
:103C5000DA0181110EC08091DB0181110AC08091CF
:103C6000DC01811106C08091DD01811102C010923A
:103C7000D801089589ED91E00E94A30E0E94A11A37
:103C80009093D6018093D50108951F93CF93DF932E
:103C90008091D5019091D6010E94AD1AAC0190910E
:103CA000D801992321F02091140130E006C0209121
:103CB00015018AE0289F900111244217530708F448
:103CC00085C08091DA01C091DB01D091DC011091B7
:103CD000DD01811107C0C11175C0D11173C011116F
:103CE00071C074C09F3F19F09F5F9093D801181660
:103CF00024F40E94CB1C8093DA018091DA0187FFC3
:103D000005C00E94CB1C81958093DA011C1624F417
:103D10000E94CB1C8093DB018091DB0187FF05C0F3
:103D20000E94CB1C81958093DB016091DA016623B0
:103D300031F1C091DB01CC2311F1062E000C770B81
:103D4000880B990B0E94BC2123E333E343E35FE339
:103D50000E9420220E9484216093DA016C2FCC0FF4
:103D6000770B880B990B0E94BC2123E333E343E3D9
:103D70005FE30E9420220E9484216093DB011D16D4
:103D800024F40E94141D8093DC018091DC0187FFE4
:103D900005C00E94141D81958093DC01111624F446
:103DA0000E94141D8093DD018091DD0187FF05C015
:103DB0000E94141D81958093DD01DF91CF911F91A9
:103DC0000C943A1E9F3F09F08FCFA0CFDF91CF9187
:103DD0001F910895E9EDF1E085E0DF011D928A95DC
:103DE000E9F71092D8011092D7010895833081F13C
:103DF00028F4813059F08230D1F00895853009F4EB
:103E000049C0B8F1863009F456C008958091150173
:103E1000262F30E0280F311D2F3F310524F4680F85
:103E20006093150108958FEF809315010895809197
:103E30001401262F30E0280F311D2F3F310524F4C7
:103E4000680F6093140108958FEF80931401089513
:103E500080911301262F30E0280F311D2F3F3105AF
:103E600024F4680F6093130108958FEF809313017A
:103E7000089580911201262F30E0280F311D2F3F29
:103E8000310524F4680F6093120108958FEF809339
:103E90001201089580911101262F30E0280F311D65
:103EA0002F3F310524F4680F6093110108958FEFBF
:103EB00080931101089580911001262F30E0280F82
:103EC000311D2F3F310524F4680F609310010895D0
:103ED0008FEF809310010895833011F128F4813021
:103EE00049F0823091F00895853081F120F18630DB
:103EF000C1F1089580911501681720F4861B809305
:103F00001501089510921501089580911401681704
:103F100020F4861B809314010895109214010895D3
:103F200080911301681720F4861B80931301089574
:103F300010921301089580911201681720F4861BD6
:103F40008093120108951092120108958091110139
:103F5000681720F4861B80931101089510921101B7
:103F6000089580911001681720F4861B809310013A
:103F700008951092100108950F931F938D3109F445
:103F80006BC008F03FC08E3009F47DC0C0F48730AC
:103F900009F46EC068F4863009F0AFC08091D0019A
:103FA000817F8E7F8093D00181E08093DF01A6C066
:103FB000883009F458C08B3009F49BC09EC086310C
:103FC00009F497C078F4803109F470C0813109F0A8
:103FD00094C00E94F51390910D0181E08927809390
:103FE0000D0187C0893109F484C08B3109F085C087
:103FF0008091D00181FB222720F991E0922790FB4C
:1040000081F94AC0853309F45BC048F4873209F46A
:1040100057C008F45AC0893209F452C06EC08334C4
:1040200038F48A3308F067C0883309F462C065C089
:10403000833409F445C0883409F05FC00E94F51349
:104040000FEF13ED20E3015010402040E1F700C0D6
:1040500000000E94FC1A4DC00E943E210E948C0E5E
:104060000E94820746C00E94B01C0E94C21C41C030
:104070009091D001892F817090FF12C0917F9E7F17
:104080009093D0013BC08091D00182FB222720F980
:1040900091E0922790FB82F98093D001992349F116
:1040A0008091D00181608093D00123C08091D001A4
:1040B00083FB222720F991E0922790FB83F9ECCF34
:1040C00061E070E080E090E010C08D5141E050E090
:1040D00060E070E08A019B0104C0000F111F221FE5
:1040E000331F8A95D2F7C901B8010E94AC170E940C
:1040F000F51381E003C08953E9CF80E01F910F9150
:10410000089580E008950C948120CF93C82F80916A
:10411000DF01813079F018F08230E9F187C0E09159
:104120000E01F0910F018081813169F0823209F036
:104130007FC009C0E0910E01F0910F0180818131B3
:1041400011F0823261F48C2F0E948320811104C00F
:104150008C2F0E94BC1F1DC081E090E01AC08C2FE4
:104160000E948120811114C0C43179F048F4CB3011
:1041700079F0C03109F060C082E08093DF0108C0AF
:10418000C93219F0C83321F057C01092DF0154C072
:1041900081E0817053C0C93289F118F5C43171F1E1
:1041A000A8F4C73009F046C08AE08093150194E175
:1041B0009093140193E0909313018093120188E08F
:1041C0008093110188E28093100134C0CE51C63033
:1041D00088F5EC2FF0E0E65DFE4F80818093DE01F4
:1041E00029C0CE34E9F020F4CB3421F56AE013C0C5
:1041F000C13579F0C235F1F461E00DC08091DE0186
:10420000882319F01092DE0115C081E08093DF0150
:1042100015C061E006C08091DE010E94F61E0AC052
:104220006AE08091DE010E946C1F04C01092DF01E1
:1042300080E004C081E002C080E0ABCFCF91089560
:10424000E1E8F0E080818860808380818160808304
:104250008FB7F89493E09093890090ED9093880045
:104260008FBF0895EFE6F0E080818260808308953B
:10427000EFE6F0E080818D7F80830895EFE6F0E047
:10428000908182E08927808308951F920F920FB654
:104290000F9211242F933F934F935F936F937F93CC
:1042A0008F939F93AF93BF93EF93FF938091E00120
:1042B0009091E10101969093E1018093E0018111D9
:1042C00003C082E00E948207E091E101E695E69555
:1042D000F0E0EA57FB4FE4918091E0018E1303C0B8
:1042E00080E00E948207FF91EF91BF91AF919F9173
:1042F0008F917F916F915F914F913F912F910F908F
:104300000FBE0F901F9018950E948B216894B111D9
:104310000C941A2208950E94FF2188F09F5798F06C
:10432000B92F9927B751B0F0E1F0660F771F881FBA
:10433000991F1AF0BA95C9F714C0B13091F00E94D4
:104340001922B1E008950C941922672F782F88273D
:10435000B85F39F0B93FCCF3869577956795B395FB
:10436000D9F73EF490958095709561957F4F8F4F6A
:104370009F4F0895E89409C097FB3EF4909580956F
:10438000709561957F4F8F4F9F4F9923A9F0F92F1B
:1043900096E9BB279395F695879577956795B79599
:1043A000F111F8CFFAF4BB0F11F460FF1BC06F5F7F
:1043B0007F4F8F4F9F4F16C0882311F096E911C091
:1043C000772321F09EE8872F762F05C0662371F0B2
:1043D00096E8862F70E060E02AF09A95660F771FC6
:1043E000881FDAF7880F9695879597F9089557FDF6
:1043F0009058440F551F59F05F3F71F04795880F53
:1044000097FB991F61F09F3F79F0879508951216E9
:1044100013061406551FF2CF4695F1DF08C0161695
:1044200017061806991FF1CF869571056105089446
:104430000895E894BB2766277727CB0197F908955D
:104440000E9433220C94A4220E94962238F00E94EB
:104450009D2220F0952311F00C948D220C94932230
:1044600011240C941A220E94F72170F3959FC1F336
:10447000950F50E0551F629FF001729FBB27F00D12
:10448000B11D639FAA27F00DB11DAA1F649F662767
:10449000B00DA11D661F829F2227B00DA11D621FB6
:1044A000739FB00DA11D621F839FA00D611D221F70
:1044B000749F3327A00D611D231F849F600D211D54
:1044C000822F762F6A2F11249F5750409AF0F1F0D7
:1044D00088234AF0EE0FFF1FBB1F661F771F881F40
:1044E00091505040A9F79E3F510580F00C948D22C9
:1044F0000C941A225F3FE4F3983ED4F386957795A7
:104500006795B795F795E7959F5FC1F7FE2B880FE5
:10451000911D9695879597F9089597F99F6780E87B
:1045200070E060E008959FEF80EC089500240A9405
:104530001616170618060906089500240A9412167E
:104540001306140605060895092E0394000C11F4B1
:10455000882352F0BB0F40F4BF2B11F460FF04C05E
:104560006F5F7F4F8F4F9F4F089597FB072E16F475
:10457000009407D077FD09D00E94CF2207FC05D018
:104580003EF4909581959F4F0895709561957F4F6A
:104590000895EE0FFF1F0590F491E02D0994AA1BDA
:1045A000BB1B51E107C0AA1FBB1FA617B70710F01E
:1045B000A61BB70B881F991F5A95A9F78095909550
:1045C000BC01CD010895F999FECF92BD81BDF89A45
:1045D000992780B50895A8E1B0E042E050E00C943E
:1045E0000623262FF999FECF1FBA92BD81BD20BDAB
:1045F0000FB6F894FA9AF99A0FBE019608950E94A0
:10460000F122272F0C94F222DC01CB01FC01F99955
:10461000FECF06C0F2BDE1BDF89A319600B40D920E
:0C46200041505040B8F70895F894FFCFC7
:10462C00200283071308EE07BA0786070101BE01B3
:10463C0028080A03140A3F4D36394704FA03C40309
:10464C008B031E03370350036903010203040506A1
:04465C000708090042
:00000001FF
